:100000000C945B000C94AD010C94DA010C94830009
:100010000C9483000C9483000C9483000C94830054
:100020000C9483000C9483000C9483000C94830044
:100030000C9483000C9483000C9483000C94830034
:100040000C9407020C9483000C94B6030C94830068
:100050000C9483000C9483000C9483000C94830014
:100060000C9483000C948300000024272A000025B0
:10007000282B000023262904040404040404040299
:100080000202020202030303030303010204081035
:100090002040800102040810200102040810200002
:1000A0000000070002010000030406000000000039
:1000B00000000000C30011241FBECFEFD8E0DEBF58
:1000C000CDBF11E0A0E0B1E0EEEBF8E002C005909A
:1000D0000D92AA30B107D9F711E0AAE0B1E001C052
:1000E0001D92A13AB107E1F710E0C6EBD0E004C0E1
:1000F0002297FE010E945904C43BD107C9F70E9410
:10010000BC000C945D040C9400008BE091E00E9414
:10011000D1008823B9F08BE091E00E94CE0080935B
:100120000A01809102010E94F902892BD1F74091C6
:100130000A0150E060E070E020E030E08BE091E008
:100140000E949801089540E855E260E070E08BE07D
:1001500091E00E94D40060E0809100010E94DB02E7
:1001600060E0809102010E94DB0264E670E080E0C2
:1001700090E00E94770208950E94A1020E94A300CD
:100180000E948500FDCF88E091E090930C01809360
:100190000B010895862F0E947E0308950E94970305
:1001A00008950E9486030895CB01BA010E94450379
:1001B00008952F923F924F925F926F927F928F920B
:1001C0009F92AF92BF92CF92DF92EF92FF920F93E6
:1001D0001F93DF93CF93CDB7DEB7A0970FB6F894F8
:1001E000DEBF0FBECDBF1C016A017B014115510569
:1001F0006105710549F4DC01ED91FC910190F081FC
:10020000E02D60E3099554C0882499245401422EBE
:1002100055246624772401E010E00C0F1D1F080D03
:10022000191DC701B601A30192010E940604F8013D
:1002300060830894811C911CA11CB11CC701B601EC
:10024000A30192010E940604C901DA016C017D013B
:10025000C114D104E104F104F1F681E0E82EF12C9F
:10026000EC0EFD1EE80CF91C3E010894611C711C8B
:10027000D501C4010197A109B1096C01C818D908B9
:1002800014C0F601EE0DFF1D60816A3010F4605D50
:1002900001C0695CD101ED91FC910190F081E02DEC
:1002A000C10109950894E108F1086E147F0449F72B
:1002B000A0960FB6F894DEBF0FBECDBFCF91DF91F1
:1002C0001F910F91FF90EF90DF90CF90BF90AF9074
:1002D0009F908F907F906F905F904F903F902F9066
:1002E0000895EF92FF920F931F93CF93DF93EC014A
:1002F0007A018B0177FF0FC0E881F9810190F081CD
:10030000E02D6DE2099510950095F094E094E11CC4
:10031000F11C011D111D2AE0B801A701CE010E94A8
:10032000D900DF91CF911F910F91FF90EF90089529
:10033000DC012115310541F4ED91FC910190F08132
:10034000E02D642F099508952A30310519F40E9493
:10035000710108950E94D90008951F920F920FB65F
:100360000F9211242F933F934F935F936F937F933B
:100370008F939F93AF93BF93EF93FF9380910D0162
:1003800090910E01892B29F0E0910D01F0910E0161
:100390000995FF91EF91BF91AF919F918F917F91BF
:1003A0006F915F914F913F912F910F900FBE0F90E2
:1003B0001F9018951F920F920FB60F9211242F9332
:1003C0003F934F935F936F937F938F939F93AF93DD
:1003D000BF93EF93FF9380910F0190911001892BB0
:1003E00029F0E0910F01F09110010995FF91EF9133
:1003F000BF91AF919F918F917F916F915F914F913D
:100400003F912F910F900FBE0F901F9018951F9244
:100410000F920FB60F9211242F938F939F93AF9348
:10042000BF938091110190911201A0911301B0919D
:1004300014010196A11DB11D809311019093120129
:10044000A0931301B09314018091150190911601AE
:10045000A0911701B09118018050904CAF4FBF4F41
:100460008093150190931601A0931701B093180182
:1004700027C08091150190911601A0911701B091AC
:10048000180180589E43A040B0408093150190937E
:100490001601A0931701B093180180911901909152
:1004A0001A01A0911B01B0911C010196A11DB11D63
:1004B0008093190190931A01A0931B01B0931C0122
:1004C0008091150190911601A0911701B09118012A
:1004D00081589E43A040B04060F6BF91AF919F917C
:1004E0008F912F910F900FBE0F901F901895EF9244
:1004F000FF920F931F937B018C018FB7F89440916B
:10050000190150911A0160911B0170911C018FBF5C
:100510002FB7F8948091190190911A01A0911B01B5
:10052000B0911C012FBF841B950BA60BB70BE816CF
:10053000F9060A071B0760F71F910F91FF90EF90D4
:100540000895789484B5826084BD84B5816084BD4B
:1005500085B5826085BD85B5816085BDEEE6F0E03C
:10056000808181608083E1E8F0E080818260808327
:10057000808181608083E0E8F0E080818160808319
:10058000E1EBF0E0808184608083E0EBF0E080814B
:1005900081608083EAE7F0E08081846080838081ED
:1005A0008260808380818160808380818068808395
:1005B0001092C1000895282F30E0C90185579F4F40
:1005C000FC01949129583F4FF9018491882381F0CF
:1005D000E82FF0E0E859FF4FE491F0E0662329F4BA
:1005E000808190958923808308958081892B8083E1
:1005F0000895482F50E0CA0181569F4FFC01249175
:10060000CA0185579F4FFC01949149585F4FFA01E9
:100610003491332319F420E030E035C0222331F146
:10062000233021F4809180008F7705C0243031F48D
:10063000809180008F7D8093800018C0213019F454
:1006400084B58F7704C0223021F484B58F7D84BDBA
:100650000DC0263021F48091B0008F7705C027307F
:1006600029F48091B0008F7D8093B000E32FF0E0FB
:10067000EE58FF4FE491F0E0808120E030E08923E4
:1006800011F021E030E0C9010895EF92FF920F933D
:100690001F937B018C0122E030E040E050E00E949B
:1006A0002804205C3D4B404F5F4FCA01B901A801AF
:1006B00097010E942804C901DA010197A109B10933
:1006C000292F3A2F4B2F552747FD5A950196A11DEB
:1006D000B11D2093C50081508093C400E1ECF0E08F
:1006E0008081806180838081886080838081806850
:1006F00080831F910F91FF90EF900895982F809124
:10070000C00085FFFCCF9093C600089580911D0125
:1007100090911E0180589F4F20911F013091200120
:10072000821B930B60E870E00E94F30308954091F0
:100730001F015091200180911D0190911E0184178D
:10074000950719F42FEF3FEF0FC0FA01EF5DFE4F51
:100750002081CA01019660E870E00E94F303909343
:10076000200180931F0130E0C90108951F920F926C
:100770000FB60F9211242F933F934F935F936F9374
:100780007F938F939F93AF93BF93EF93FF9340918A
:10079000C600E0911D01F0911E01CF01019660E8B5
:1007A00070E00E94F3039C0180911F019091200151
:1007B0002817390739F0EF5DFE4F408330931E0153
:1007C00020931D01FF91EF91BF91AF919F918F9168
:1007D0007F916F915F914F913F912F910F900FBE3D
:1007E0000F901F90189597FB092E07260AD077FDCA
:1007F00004D049D006D000201AF4709561957F4F3F
:100800000895F6F7909581959F4F0895A1E21A2ECD
:10081000AA1BBB1BFD010DC0AA1FBB1FEE1FFF1FA4
:10082000A217B307E407F50720F0A21BB30BE40BF4
:10083000F50B661F771F881F991F1A9469F760953B
:100840007095809590959B01AC01BD01CF010895F5
:1008500097FB092E05260ED057FD04D0D7DF0AD00E
:10086000001C38F450954095309521953F4F4F4FDF
:100870005F4F0895F6F790958095709561957F4F3D
:100880008F4F9F4F0895AA1BBB1B51E107C0AA1FA2
:10089000BB1FA617B70710F0A61BB70B881F991F21
:1008A0005A95A9F780959095BC01CD010895EE0F5A
:0E08B000FF1F0590F491E02D0994F894FFCFFE
:0A08BE000600070000000000CA0059
:00000001FF
